:100000000004001001010000D5000000D90000002C
:1000100000000000000000000000000000000000E0
:10002000000000000000000000000000BD0500000E
:10003000000000000000000075050000250500001C
:1000400045010000450100000000000045010000DE
:100050004501000045010000000000000000000014
:100060004501000045010000450100004501000078
:1000700045010000450100000000000045010000AE
:100080000000000000000000000000000000000070
:100090000000000000000000000000000000000060
:1000A0004501000045010000450100004501000038
:1000B0004501000045010000450100004501000028
:1000C000FC08000000000010040000000400001004
:1000D0004002000000B5FEE700B5FEE710B50023C2
:1000E00002E01C58043310C19342FAD310BD10B57E
:1000F000031C002200E004C31C1A8C42FBD310BD79
:1001000038B50D4C0D4D05E020686168A2680C34CF
:10011000FFF7E4FFAC42F7D305E0206861680834DC
:10012000FFF7E5FF00E0064DAC42F6D300F044FBDC
:1001300000F064FBFEE7C046C0000000CC000000F9
:10014000D400000000B5FEE710B5A02280231206FF
:100150009B010124D1588440201C0843D05010BD7D
:10016000F7B5304D4022EB6F2F4C1343EB67EB6F2D
:1001700080221343EB6762682C4B4D211340636070
:1001800062688023DB0013436360294A294B49429C
:100190001A60E022520099501120FFF7D5FF10207D
:1001A000FFF7D2FF0720FFF7CFFF234B2349082299
:1001B00001271F60CA67E86F8021C9010143E96711
:1001C000616805269143616061680A4362601C4A68
:1001D0001C4C1968106826601B68002B21D000F0A9
:1001E00011FBE12105094902281C00F00BFB164B0D
:1001F000FF22013820621A601868216A1B68C01942
:100200000193CB19E12149025943684300F0FAFAFE
:10021000019AD343C0180D4B1860A66023681F4392
:100220002760F7BD0480044000800440FFFBFFFF0F
:100230000400FFFF00C000409480044004E100E09F
:100240000000001000400640F0800440F4800440AC
:1002500010B5A023802480211B06A4024902882215
:10026000002800D18A2292019C50995080219950F7
:1002700010BD000000B5044B9A68510701D5D86144
:1002800001E00120404200BD0040064000B5044BA3
:100290009A68D10701D5586901E00120404200BDAC
:1002A0000040064010B5041C08E000F03EFA20783B
:1002B000FFF7E0FF23789842F7D101342378002B31
:1002C000F5D110BDF7B50025124E2F1CFFF7DEFF4C
:1002D000041E12DB002D05D10F48FFF7E3FF0F4886
:1002E000FFF7E0FF0D2C01D10B4802E001A80470DC
:1002F0004770FFF7D7FF0A4D08E0002D02D0013DFF
:10030000002D03D1301CFFF7CDFF002500F00DFAC2
:10031000DCE7C04690080000BC0800007808000038
:10032000F301000008B50120FFF792FFFA2040001A
:1003300000F0F8F90020FFF78BFFFA20400000F0F2
:10034000F1F9F0E708B5FFF70BFF00F0D7F901204E
:1003500006490A2200F0A2F902200549142200F001
:100360009DF900F069F9002008BDC0462503000092
:10037000C502000000B5031C30331A0419061143EE
:10038000054A1943C0011B02194310180023C1502C
:100390000433802BFBD100BD04000010704700B572
:1003A000002901D106E0181C8368002BFBD1816075
:1003B00048608B6000BD00B58368002B07D09A6849
:1003C0008260002A00D0506000225A609A60181C97
:1003D00000BD00B50DE088420BD142688368002A59
:1003E00000D09360002B00D05A60002343608360EC
:1003F00002E080680028EED100BD38B50D1C00E099
:10040000201C8468A847002CFAD138BD10B5064AD4
:10041000064B072004211468844314601C698C4334
:100420001C6130BFF7E7C0460000024000ED00E06D
:1004300070B5002816DAC0B20F230340083B134AF8
:100440009B089B009B18032210409040FF225D6890
:10045000141C84408901A5430A408240281C104393
:10046000586011E003248208094B2040C032A040AC
:100470009200FF24D558261C86408901B5430C40C4
:100480008440281C2043D05070BDC04618ED00E0C9
:1004900000E100E010B50369011C002B0DD1094CEF
:1004A000201C3030FFF795FF011E08D00123201CCF
:1004B0000B731030FFF773FF01E0013B0361002075
:1004C00010BDC0468401001010B5144CE36D002B24
:1004D00006D00023201CE36530301149FFF78DFF63
:1004E000E168002911D00B7B012B05D0002B02D035
:1004F000022B04D008E0FEE7201C103001E0201C95
:100500003030FFF74CFF00E0FEE7044C201C1030B9
:10051000FFF751FF002800D0E06010BD84010010FB
:100520009504000000B5104B104A996D0131996592
:10053000914204D900219965596D01315965DB68F3
:10054000D9690131D961914204D90022DA619A69ED
:1005500001329A61044B0122DA65054B8022596809
:1005600052050A435A6000BD84010010E7030000F1
:1005700000ED00E0EFF30982203AF0C244464D4618
:1005800056465F46F0C2203A0B49C868026000B583
:10059000FFF79AFF01BC86460749C8680268103217
:1005A000F0CAA046A946B246BB46203AF0CA10326D
:1005B00082F309887047C046840100101B4A5060CE
:1005C0001A4A916070460421084202D0EFF3098173
:1005D00001E0EFF308818A69023A1078134A10604B
:1005E00080B484B06F46124B1A78012A14D0002AC6
:1005F0000DD0802A16D10D49C868026882F3098897
:1006000004217046084386460A4B596807E0DA68B9
:100610005B68022111731361064B802259685205F1
:100620000A435A6004B080BC7047C0468401001081
:100630008401001000ED00E010B500F079F8144BD3
:10064000FA211868890000F0DDF8124C013860606A
:10065000012040420321FFF7EBFE0023A3600520A9
:100660000723236040428021FFF7E2FE0120404241
:10067000C021FFF7DDFE02204042FF21FFF7D8FE38
:10068000054B802212061A6080DFC046FEE7C04696
:100690000000001010E000E000E100E070B5154C33
:1006A0004301E418151C0E1CFFF764FE031C4033C5
:1006B00023600122002322736360A36065610366E7
:1006C00043670D4D80235B04C3672B6D4266022296
:1006D00082668667002B03D160302060EC6004E006
:1006E000281C1030211CFFF75AFE2B6D01332B659F
:1006F00070BDC046E40100108401001010B5074C25
:10070000201C1030FFF74AFE201C3030FFF746FE59
:10071000002003490122FFF7C1FF10BD8401001032
:100720000D04000000DFC046704701DFC04670477F
:1007300070B51D4D00206B6ADB051B0F013B0E2BB6
:1007400002D81A4A9B009858696A2A6F0326164BEA
:100750003240174C022A0CD0B24212D0012A03D1E7
:100760001B6C1E40022E01D0124B00E000232360C0
:1007700012E01F2319404900023100F043F82060C5
:100780000AE0196C0A40022AF0D09B681F20094930
:100790001840013041432160054CA96F206800F0EA
:1007A00031F8206070BDC04600800440C0080000E1
:1007B00000000010001BB70010B50D4A0D48D16FA6
:1007C0000D4B0143D16700221A6401225A64101CA8
:1007D0005C6C094901220442FAD0002008674A678C
:1007E000596F1142FCD0044B01229A6710BDC046DC
:1007F00004800440800004000080044008B5FFF736
:10080000A1FD08BD002931D00122D207030901E072
:10081000090112099942FBD9430801E04900520835
:100820009942FBD900E04908401A07D35241FAD354
:1008300001461046704749084018F7D29218FAD37B
:100840004018014610467047CB0F00D049420210B5
:1008500000D54042534008B5FFF7D4FF0CBC5210FE
:1008600000D34042002A00D549421847F4460020F0
:1008700000F001F860477047596561682E2049749F
:10088000277320796F7572207475726E2E0D0A00B1
:1008900054686520717569636B2062726F776E2092
:1008A000666F78206A756D7073206F76657220743C
:1008B0006865206C617A7920646F672E0D0A0000EC
:1008C00020A1070000350C00E0C81000C05C150036
:1008D000006A180040771B0080841E00C091210030
:1008E000009F240040AC2700E032290020402C006B
:0C08F000604D2F0000D4300040E13300C8
:0408FC00001BB70026
:0400000300000101F7
:00000001FF
